:020000040800F2
:10D8000020491F48214A08601F4909681160214AC0
:10D810001F491160214A20491160224A20491160A4
:10D82000224A21491160234A21491160234A224991
:10D830001160244A22491160244A23491160244975
:10D84000244A09681160254A23491160254A244960
:10D850001160264A24491160264A25491160274A49
:10D8600025491160274A26491160284A2649116036
:10D87000284A2749116028490860284908607047EC
:10D8800049300008B4010020C8020020E401002053
:10D890004B300008B801002061EA0008BC010020FC
:10D8A000D7E90008C8010020ADE70008C00100204A
:10D8B00093E70008C40100208FE70008B0010020B2
:10D8C00051E70008F001002033E60008A001002025
:10D8D00008030020DC01002033DF0008E001002005
:10D8E00007DF0008CC010020E7DE0008A4010020CB
:10D8F000F7DB0008AC0100209FDB0008D00100200E
:10D900004FDA0008A801002011DA0008D401002035
:10D9100021D90008E8010020D8010020EC010020F6
:10D92000FE48017B002919D0FD490A78002A15D14B
:10D9300001220A70FB49007D0968142805D01528CA
:10D9400006D0162807D0F8480847F7482430FBE7E8
:10D95000F5481830F8E7F4480C30F5E7704710B593
:10D96000F248F34C00782268142805D00A2805D024
:10D97000142806D91C2107E01C2100E026210120E3
:10D980000BE00A2802D9262101209047E9480068C7
:10D990008047E948226801780120BDE8104010471F
:10D9A00070B5DE4DE2480024697B026821B12D216B
:10D9B000002090476C7329E0A87B20B12A21002029
:10D9C0009047AC7322E0E87B20B12E2100209047E5
:10D9D000EC731BE0287C20B12B21002090472C7495
:10D9E00014E0687C20B12F21002090476C740DE07A
:10D9F000A87C20B12C2100209047AC7406E0E87C84
:10DA0000002804D0302100209047EC74012070BD24
:10DA10002DE9F047C94EC54D30682C788047C8487D
:10DA2000012780460770DFF81C930AE0D9F8001040
:10DA3000782088472C70FFF792FF3068804788F87D
:10DA40000070FFF7ADFF0128F0D0BDE8F087BF49B7
:10DA500010B5BD480860B448BD49001FB44C08600B
:10DA6000BC4903200870B848BB49001F08600C215E
:10DA70002268012090470321226801209047B7487F
:10DA8000B7490078801C0870B6490120087010BDA5
:10DA900010B5B54CA448216800788847A248216891
:10DAA0000C3000788847A0482168183000788847F3
:10DAB0009D4821682430007888479D4C142100201F
:10DAC000226890471521226800209047162122687D
:10DAD0000020904722681721BDE810400020104721
:10DAE000A248002101608D494A7B0AB101220260EF
:10DAF0008A7B1AB1026842F002020260CA7B1AB144
:10DB0000026842F0040202600A7C1AB1026842F024
:10DB1000080202604A7C1AB1026842F010020260F8
:10DB20008A7C1AB1026842F020020260C97C002996
:10DB300003D0016841F040010160704700B5FFF774
:10DB4000CFFF764989480A7A1AB1026842F080020A
:10DB50000260CA791AB1026842F4807202608A795E
:10DB60001AB1026842F4007202604A791AB102687E
:10DB700042F4806202600A791AB1026842F40062DB
:10DB80000260CA781AB1026842F480520260897851
:10DB9000002903D0016841F40051016000BD7448C0
:10DBA00010B5007880B9FFF7C9FF72485B496F4A2A
:10DBB0000078012811D0022814D00328087D16D03F
:10DBC00008766D4910680860FFF762FF6B48664988
:10DBD00000780968BDE810400847087D4875684925
:10DBE0001068F0E7087D887566491068EBE7C8752E
:10DBF00065491068E7E7654910B51D20087064495C
:10DC00002620664A087063491C20664B08706249EA
:10DC10000020664C087048708870C87008713C21FC
:10DC200011605F4A012111701E221A705E4A0A2398
:10DC300011703A4917220A7523700B23CB72504B8F
:10DC40001860504B4A7518604F4B8A7518604A4BE4
:10DC5000CA7518600A7610BD554A10B512211268AF
:10DC6000012090472D4800218170C17001714171E0
:10DC70008171C17101724F48324900780968BDE86D
:10DC80001040143008472DE9F0414B4A092100208B
:10DC900012689047284D264E2A4F00243268297872
:10DCA000012090473968462088473268297800204B
:10DCB0009047396846208847641CE4B2042CEDD3B1
:10DCC000BDE8F0812DE9F041144E1B4D0024707B1E
:10DCD00030B1B07820B92D202870FFF7D4FF7473CD
:10DCE000B07B134F50B1F07840B92A202870FFF76D
:10DCF000CAFFB47327213A6801209047F07B30B106
:10DD0000307920B92E202870FFF7BDFFF473307CE6
:10DD100010B1707900B951E059E000003D070020D2
:10DD2000BB030020300300206C070020CC03002040
:10DD300010030020E4020020DA0300207403002016
:10DD4000D00300206C0300205A070020CC050020DF
:10DD5000D0050020A405002028020020E0030020B8
:10DD6000DF0300207E030020EC020020700400206E
:10DD7000C9030020EE0300206C04002004050020ED
:10DD8000600400206404002068040020CD0300200B
:10DD9000CE030020CF0300207C0400205802002086
:10DDA000DC030020DD030020B7030020B1030020C6
:10DDB0000403002039020020240300202B202870B7
:10DDC000FFF761FF347428213A6801209047707C86
:10DDD00030B1B07920B92F202870FFF754FF747448
:10DDE000B07C50B1F07940B92C202870FFF74BFF80
:10DDF000B47429213A6801209047F07C002807D0AC
:10DE0000307A002804D130202870FFF73CFFF474EA
:10DE100056E770B5FF4DFE4C00202A68217D9047E3
:10DE2000207D14280BD0401E2075E07A2070FA481F
:10DE3000217D01702A68BDE8704001201047F74835
:10DE4000007828B1F649002008702A681A21904706
:10DE5000FFF738FF17202075FFF7FEFEE5E710B546
:10DE6000EB4CED48217D0170207B00B3E948A37A9B
:10DE7000026823B1002090470020A0720BE001202F
:10DE8000A072207828B1012090472078401E207091
:10DE900001E0FFF7BEFF207DE24A142814D01528C8
:10DEA00014D0162814D00821126800209047207D35
:10DEB000DD4914280ED015280FD0162810D0DB48C5
:10DEC0000968BDE8104008470521EDE70621EBE7AA
:10DED0000721E9E7D5482430F2E7D4481830EFE7C6
:10DEE000D2480C30ECE710B51E2808D01F2806D009
:10DEF000202804D0212802D04FF0FF3010BDFFF7BA
:10DF0000AEFF002010BDC74A10B5042112680020E2
:10DF10009047C849C648096800788847BD4C0C211D
:10DF200000202268904722681721BDE81040012098
:10DF300010472DE9F047C04EDFF80083C04C317820
:10DF400098F80000BF4DDFF8009381420FD122689E
:10DF5000BEA1012090472268BEA107209047AF4F85
:10DF600038782870D9F8000080472878387098F8F9
:10DF700000003178401C81420FD12268B7A10120F6
:10DF800090472268B7A107209047B84C20782870A6
:10DF9000D9F8000080472878207056E52DE9F04137
:10DFA000B34F9B4E9B4C38684FF00105410607D597
:10DFB000F57480F0400038603021226801209047DD
:10DFC0003868810605D5B57480F020002C213860B2
:10DFD00000E029212268012090473868C10607D552
:10DFE000757480F0100038602F212268012090475E
:10DFF0003868010705D5357480F008002B2138609A
:10E0000000E028212268012090473868410707D5A1
:10E01000F57380F0040038602E21226801209047BB
:10E020003878800709D5B5732A21226801209047E6
:10E03000386880F00200386003E027212268012060
:10E0400090473878C00706D075732268BDE8F04164
:10E050002D210120104733E62DE9F0414FF47A7865
:10E06000844D704E844F854C09E0296840468847AE
:10E070000B2132680020904739687D20884720684E
:10E08000401E2060401CF0D11AE62DE9F041DFF877
:10E0900080817B48012488F80C4001787748052965
:10E0A00001D2052100E003210160FFF7D5FF754E85
:10E0B000754F584D307810B938781D2811D3FFF7B7
:10E0C0000FFD724800688047FFF768FF1B212A6830
:10E0D00000209047002030703C701D212A680120EC
:10E0E000904730212A680120904788F8134088F82B
:10E0F0000D402D212A68012090475F496448096836
:10E1000000688847634A012100201268BDE8F04199
:10E110001047614810B500684FF47A7190FBF1F236
:10E1200001FB12013F48B1F5617F026801DB072165
:10E1300000E00C21002090474E4964200968BDE8AA
:10E140001040084770B54C4D4C4C04E0FFF7E1FF20
:10E150002968502088472068401E2060401CF5D167
:10E1600070BD464905200860ECE729490120087385
:10E170003448007800B1F4E74049022008606BE7BA
:10E1800010B5234C2F49234AE07C087030211268D7
:10E1900001209047FFF7E9FF002020730120E07481
:10E1A00010BD70B51A4D27491A4CA87C08702C2157
:10E1B0002268012090472921226800209047FFF71C
:10E1C000D4FF0120A87470BD124A10B52E21126828
:10E1D000012090470E4C1B49E07B0870FFF7C5FFFC
:10E1E0000120E07310BD70B50A4C2A21012022687D
:10E1F0009047074D1349A87B0870FFF7B6FF012031
:10E20000A8732268BDE87040272100201047000055
:10E210003D07002010030020DA0300202D0200201B
:10E220008605002024030020300300206C07002016
:10E230008C040020EC020020DE030020E00300201C
:10E24000FC020020B2030020E8020020526F772079
:10E2500045420000726573657420000020526F779C
:10E260002031000053706563696C00002C020020AF
:10E2700070040020440300206C03002044040020AC
:10E280003302002097050020CC030020D401002099
:10E2900050040020040300203804002010B5F74C7F
:10E2A000F749607B0870FFF760FF01206073002072
:10E2B000F44A20732D211268BDE810400120104758
:10E2C00070B5EE4DA878002847D0E878002844D0F3
:10E2D0002879002841D0687900283ED0A879002804
:10E2E0003BD0E879002838D0287A002835D0287D1E
:10E2F0000124E44E172820D0314616280A6828D079
:10E30000152804D3E0481B21047001209047FFF733
:10E31000BFFBDF49172028750968DC488847FFF7ED
:10E320009BFCDC4A0E21002012689047DA494FF42A
:10E3300096700968BDE870400847D848007810B169
:10E34000D74800688047D7481921047001203268F7
:10E35000DCE7D5481A210470D7E770BDC74A10B56D
:10E3600001211173002814D1D0480178D048052923
:10E3700001D2042100E002210160FFF76DFEF9F7F0
:10E3800064F9CC49C8200860C3490968BDE8104059
:10E39000084710BD10B5B94CA078FFF7DFFF01208A
:10E3A000A070BDE810408BE7C14914200860C9E6A1
:10E3B000B24901200873B248007800B1D1E6F3E712
:10E3C00070B5B04C05460146226801209047B2491D
:10E3D000C8200968884729462268BDE870400020A7
:10E3E00010472DE9F041A54CA54D0126207C60B9D0
:10E3F0002870FFF7BAFEA34F267428213A68002040
:10E4000090472B213A68012090471020FFF7D8FF52
:10E41000A07818B12E70BDE8F041C9E7002028703F
:10E42000FFF7C6FFBDE8F041B4E7A34810B50068A8
:10E43000642190FBF1F201FB1200A0495A28086008
:10E4400094490A6808D00D21002090479C490A2071
:10E450000968BDE8104008470C21F5E710B50E200B
:10E46000FFF7AEFF8548864940790870BDE8104047
:10E470009EE710B5FFF7F2FF8B4C207800280AD0FA
:10E4800090480068804700207E4A20701A21126858
:10E49000BDE81040104710BD70B5784C784D607CD9
:10E4A00020B92870FFF761FE012060741320FFF788
:10E4B00087FF207A2870FFF77BFF724A2F21012007
:10E4C0001268BDE87040104710B51320FFF778FFC1
:10E4D0006A486B49007A0870BDE8104068E710B5DB
:10E4E0000F20FFF76DFF65486549C0790870BDE8EA
:10E4F00010405DE710B51220FFF762FF5F486049EA
:10E5000080790870BDE8104052E710B51120FFF780
:10E5100057FF5A485A4900790870BDE8104047E74C
:10E5200010B50D20FFF74CFF54485549C0780870CE
:10E53000BDE810403CE7514910B501200873504830
:10E54000007810B1BDE810400BE6FFF72DFF5C49E5
:10E550004FF4FA6009688847BDE81040F9F775B8CC
:10E5600010B51020FFF72CFF44484549807808700B
:10E57000FFF7E1FF4B4C2078002809D0414A1921D0
:10E5800000201268904746480068804700202070AD
:10E5900010BD464810B5007805280BD248494FF405
:10E5A0007A70096888473B4A0B2100201268BDE851
:10E5B00010401047BDE81040ABE510B52F4C207A55
:10E5C000FFF7CCFE01202072BDE8104078E610B5C0
:10E5D0002A4CE079FFF7C2FE0120E071BDE810404F
:10E5E0006EE610B5254CA079FFF7B8FE0120A071AA
:10E5F000BDE8104064E610B5204C6079FFF7AEFE30
:10E6000001206071BDE810405AE610B51B4C20791E
:10E61000FFF7A4FE01202071BDE8104050E610B5C0
:10E62000164CE078FFF79AFE0120E070BDE810403C
:10E6300046E610B526286ED2DFE800F01316191C46
:10E6400046494C4F87875255585B5E6164678787A0
:10E650008787876A8787876E87877174777A7D80D7
:10E660008783FFF797FE6EE0FFF7D9FF6BE0FFF7B8
:10E67000CCFF68E0FFF7BFFF65E000003D0700202A
:10E68000B203002010030020970500206C07002033
:10E6900030030020240300206C0300202C02002003
:10E6A000D8020020980500208605002033020020B3
:10E6B00044040020540400203804002048040020B2
:10E6C00044030020C0020020FFF78BFF3BE0FFF770
:10E6D0007EFF38E0FFF771FF35E0FFF75AFF32E0C9
:10E6E000FFF73EFF2FE0FFF71BFF2CE0FFF70DFFCA
:10E6F00029E0FFF7B3FE26E0FFF7FCFE23E0FFF77B
:10E70000EEFE20E0FFF7E0FE1DE0FFF7C5FE1AE099
:10E71000FFF7AFFE17E018E0FFF787FE13E0FFF703
:10E7200060FE10E0FFF7BAFD0DE0FFF75CFD0AE0C8
:10E73000FFF74AFD07E0FFF734FD04E0FFF720FD97
:10E7400001E0FFF7A2FC002010BD4FF0FF3010BD2C
:10E7500070B5F24CF24DF34E207878B1F248007B60
:10E7600020B9F24A0F21002012689047307818B182
:10E7700004212A6801209047002006E0307818B173
:10E7800004212A68002090470120207070BDFFF707
:10E790007FB9E74910B509684FF4FA708847E54A30
:10E7A000092100201268BDE81040104770B5E24C06
:10E7B0004C202168884708B1012070BD21682520C0
:10E7C0008847DE4DDE4CDF4E48B1DA4A0121002099
:10E7D00012689047052005E02168884712E03078EC
:10E7E00028B1401E3070287870B1D748F4E72878F7
:10E7F00040B1D84CD5A10120226890472268D6A10B
:10E8000007209047002070BDD548E5E770B5D54E8C
:10E81000C54D4FF001043088800407D5AC7010203E
:10E82000FFF7CEFD306880F4005030603088C004BF
:10E8300007D5EC700D20FFF7C3FD306880F48050E1
:10E8400030603088000507D52C711120FFF7B8FD26
:10E85000306880F4006030603088400507D56C7106
:10E860000E20FFF7ADFD306880F4806030603088A6
:10E87000800507D5AC711220FFF7A2FD306880F447
:10E88000007030603088C00507D5EC710F20FFF7AD
:10E8900097FD306880F4807030603078000607D5CE
:10E8A0002C721320FFF78CFD306880F08000306000
:10E8B000FFF774FB0020306070BD2DE9F05FAA4EB9
:10E8C000AA4F4FF0170BAA4986F800B04FF0000985
:10E8D000552087F800900125DFF898A2904CDFF8CA
:10E8E0004C82086027E0387828B3DAF800008047C7
:10E8F00022683178012090472D212268012090471D
:10E900002A212268012090472E2122680120904769
:10E910002B212268012090472F2122680120904757
:10E920002C21226801209047302122680120904745
:10E9300087F8009039E09048006880472D212268D0
:10E94000002090472A212268002090472E2122682B
:10E95000002090472B212268002090472F21226819
:10E96000002090472C212268002090473021226807
:10E97000002090471421226800209047152122682A
:10E980000020904716212268002090471721226816
:10E990000020904722683178012090473078142871
:10E9A00016D0401E3070012038700621D8F80020A3
:10E9B000002090476D1CEDB20A2D94D90421D8F89F
:10E9C000002000209047DAF80000BDE8F05F004723
:10E9D00086F800B0E7E770B5544A082100201268B5
:10E9E0009047FFF76AFFFFF737F964485D494E4CDF
:10E9F00000784B4D01281ED0022823D0032828D0B0
:10EA0000207E20755E480068086008212A68012081
:10EA10009047FFF7FBFE5B48006880472A68217D2E
:10EA2000012090471D212A68012090475648006820
:10EA3000BDE870400047607D20755448006808605C
:10EA40000521E3E7A07D2075514800680860062194
:10EA5000DCE7E07D20754F48006808600721D5E7B6
:10EA60003149012200204A708870C87008714871CD
:10EA70008871C871087248738873C87308744874C1
:10EA8000264B8874C8741870434B1870434B4A72F5
:10EA90008A721870424B1870424B08731A70424BBE
:10EAA0001870424B1860CB7A0B7041490A7041498B
:10EAB0000A70414908704149086041490A7041495A
:10EAC0000A7041490870414908604149087041494C
:10EAD00008607047154A0F210020126810473E4811
:10EAE00010B5006880472148007800280CD01348F2
:10EAF0000078002808D039480078022804D1384826
:10EB00000068BDE81040004710BD7047704710B561
:10EB1000FFF7D3FEBDE81040FFF79EB88705002041
:10EB200010030020C70300203D070020240300201D
:10EB30006C0300200403002064030020C2030020B3
:10EB400030030020EF030020980300202020202025
:10EB50006E6F0000FC02002062616C6C732000008C
:10EB6000A403002070040020DA030020B203002078
:10EB700054040020DC02002014030020EE030020D7
:10EB80006C040020F0020020C4010020600400207A
:10EB90006404002068040020BB03002097050020C7
:10EBA00098050020B4030020B50300204C04002089
:10EBB000CC030020D0030020BC0300209C050020D3
:10EBC000ED03002091050020C503002074040020FF
:10EBD00099050020C8050020C0010020F503002091
:04EBE00038030020D6
